:100000000C945A000C9477000C9477000C947700B1
:100010000C9477000C9477000C9477000C94770084
:100020000C9477000C9477000C9477000C94770074
:100030000C9477000C9485040C9477000C94770052
:100040000C944C050C9477000C9477000C9477007A
:100050000C9477000C9477000C9477000C94770044
:100060000C9477000C947700000024272A000025C8
:10007000282B000023262904040404040404040299
:100080000202020202030303030303010204081035
:100090002040800102040810200102040810200002
:1000A0000000070002010000030406000000000039
:1000B0000000000011241FBECFEFD4E0DEBFCDBF93
:1000C00011E0A0E0B1E0E0E7F5E102C005900D929B
:1000D000A430B107D9F711E0A4E0B1E001C01D924E
:1000E000A03DB107E1F70E9496030C94B70A0C9467
:1000F00000008EBD0DB407FEFDCF8EB59927089583
:10010000E82FFF2783E0EE0FFF1F8A95E1F7EC5FF2
:10011000FE4FE60FF11D40830895E82FFF2793E07F
:10012000EE0FFF1F9A95E1F7EC5BFE4FE60FF11D16
:1001300040830895E82FFF2723E0EE0FFF1F2A9545
:10014000E1F7EC57FE4FE60FF11D408308950F9342
:10015000A82FBB27772733E0AA0FBB1F3A95E1F7FB
:10016000FD01EC5FFE4FE60FF71F4083FD01EC5BE6
:10017000FE4FE60FF71F2083AC57BE4FA60FB71FE9
:100180000C930F910895CF93DF93582F20E030E028
:100190000BC059936D9341938F5F8830D1F72F5FD8
:1001A0003F4F2830310589F0C90173E0880F991F4E
:1001B0007A95E1F7EC01CC5FDE4FDC01AC5BBE4F22
:1001C000FC01EC57FE4F80E0E4CFDF91CF91089522
:1001D0004F925F926F927F928F929F92AF92BF9257
:1001E000CF92DF92EF92FF920F931F93D82EC62EDD
:1001F000CA0168E671E00E941C0A7C016CE370E0B1
:100200000E941C0A882777FD8095982F0E94E2089B
:100210004B015C010027F7FC0095102FC801B701C6
:100220000E94E20820E030E040E752E40E944708E4
:10023000A50194010E94E2079B01AC0160E070E01F
:1002400080E89FE30E94E2077B018C019B01AC01E7
:1002500060E070E080E89FE30E94E2072B013C0130
:1002600020E030E040E050E0C501B4010E941D09EB
:10027000882339F45301420160E070E080E89FE395
:1002800016C020E030E040E85FE3C501B4010E9401
:100290001D098823B9F4C801B7010F2EF0E08F2E95
:1002A000F0E09F2EF0E8AF2EFFE3BF2EF02D0F2ED3
:1002B000F0E04F2EF0E05F2EF0E06F2EF0E07F2EAA
:1002C000F02D5BC020E030E040E050E4C501B40117
:1002D0000E941D09882379F460E070E080E090E0DE
:1002E0000F2EF0E08F2EF0E09F2EF0E8AF2EFFE310
:1002F000BF2EF02D42C020E030E040E450E4C501C4
:10030000B4010E941D09882339F44701580160E0B7
:1003100070E080E090E016C020E030E040E850E47B
:10032000C501B4010E941D098823B9F4C301B201BB
:100330000F2EF0E08F2EF0E09F2EF0E0AF2EF0E0D9
:10034000BF2EF02D0F2EF0E04F2EF0E05F2EF0E8E4
:100350006F2EFFE37F2EF02D10C02701380160E0E3
:1003600070E080E89FE30F2EF0E08F2EF0E09F2EEC
:10037000F0E0AF2EF0E0BF2EF02D0D2D1127DD2483
:10038000A3E0000F111FAA95E1F7F4E0EF2EF1E0D2
:10039000FF2EE00EF11EEC0CFD1C20E030E048EFDB
:1003A00051E40E949A090E94B408F7016083E4E4D2
:1003B000EE2EE1E0FE2EE00EF11EEC0CFD1C20E026
:1003C00030E048EF51E4C501B4010E949A090E944F
:1003D000B408F70160830C571E4F0C0D1D1D20E063
:1003E00030E048EF51E4C301B2010E949A090E9433
:1003F000B408F80160831F910F91FF90EF90DF9098
:10040000CF90BF90AF909F908F907F906F905F90B4
:100410004F900895DF92EF92FF920F931F93CF9327
:10042000DF937C0100E010E00EC0A7016C2F8D2D42
:100430000E94E8002196C830D105B9F70F5F1F4F21
:100440000830110521F0D02EC0E0D0E0EECFDF91D2
:10045000CF911F910F91FF90EF90DF900895FF9241
:100460000F931F93CF93DF93F82E8B01C0E0D0E062
:10047000A8016F2D8C2F0E94E8002196C830D1056D
:10048000B9F7DF91CF911F910F91FF900895FF92DF
:100490000F931F93CF93DF93F82E8B01C0E0D0E032
:1004A000A8016C2F8F2D0E94E8002196C830D1053D
:1004B000B9F7DF91CF911F910F91FF9008958CB5FF
:1004C00080658CBD8CB58C7F8CBD8DB58EB58DB5A2
:1004D0008E7F8DBD0895E1E8F0E080818D7F80837F
:1004E0008081856080838081877E8083E0E8F0E082
:1004F00080818C7F8083EFE6F0E080818160808363
:100500008FEC9EEF909385008093840078940895FB
:10051000AF92BF92CF92DF92EF92FF920F931F9311
:1005200068E671E080E090E00E9423075B016C01C7
:1005300068E070E080E090E00E9423077B018C017E
:1005400068E070E080E090E00E942307DC01CB01CE
:10055000A5016E2D0E94E8001F910F91FF90EF9072
:10056000DF90CF90BF90AF900895EF92FF920F93DE
:100570001F93CF93DF93C0E0D0E0EE24FF248701E8
:10058000C801B7010E94E2080E94AF08DC01CB015C
:100590000E940A0264E070E080E090E00E94FC05A6
:1005A000239683E090E0A0E0B0E0E80EF91E0A1F79
:1005B0001B1F91E0C836D90719F7DF91CF911F9122
:1005C0000F91FF90EF90089587E00E9447068823DF
:1005D00059F48091C6019091C70101969093C7018B
:1005E0008093C60161E001C060E084E00E9497064C
:1005F0002091C6013091C7014091C4015091C501BD
:10060000A42FBB27822F8150992763E0AA0FBB1F1D
:100610006A95E1F7FD01EC5FFE4FE80FF91F1082CC
:10062000FD01EC5BFE4FE80FF91F1082AC57BE4F87
:10063000A80FB91F1C922830310554F01092C70141
:100640001092C6014F5F5F4F5093C5014093C401A4
:100650008091C4019091C501089724F01092C501C2
:100660001092C401A091C401BB278091C6019927B3
:1006700023E0AA0FBB1F2A95E1F7FD01EC5FFE4FB7
:10068000E80FF91F20E22083FD01EC5BFE4FE80F2D
:10069000F91F2083AC57BE4FA80FB91F2C936AE0F7
:1006A00070E080E090E00E94FC0508958BE292E00B
:1006B0000E94780761E084E00E94260660E087E0FF
:1006C0000E94260661E087E00E94970661E08DE0C7
:1006D0000E94260661E08AE00E94260661E08BE027
:1006E0000E94260660E08CE00E94260661E089E018
:1006F0000E94260660E08AE00E94970660E08BE098
:100700000E94970660E08DE00E9497060E945F02BB
:100710006AE070E080E090E00E94FC0540E060E06C
:1007200080E00E94C3000E946B0208950E94C205EF
:100730000E9456030E94E402FDCFCF93DF939927D6
:1007400073E0880F991F7A95E1F7EC01CC5FDE4FDB
:10075000DC01AC5BBE4FFC01EC57FE4F80E06993BF
:100760004D9321938F5F8830D1F7DF91CF9108951A
:100770008F929F92AF92BF92CF92DF92EF92FF92B1
:100780000F931F93CF93DF93982E862E5A019927AC
:10079000F3E0880F991FFA95E1F7E4E0EE2EE1E02F
:1007A000FE2EE80EF91E8C010C5B1E4FEC01CC579F
:1007B000DE4FCC24DD24882D99270C2C02C0959582
:1007C00087950A94E2F780FF06C0A5016C2D892D5C
:1007D0000E94E80005C0F7011082F801108218821B
:1007E0000894C11CD11C0894E11CF11C0F5F1F4F21
:1007F0002196F8E0CF16D104F1F6DF91CF911F9149
:100800000F91FF90EF90DF90CF90BF90AF909F90AF
:100810008F9008950F931F93CF93DF9300E010E024
:100820003DC049934D9341938F5F8830D1F72F5F3F
:100830003F4F2830310509F564E070E080E090E03A
:100840000E94FC050F5F1F4F00321105E1F126C029
:1008500019931D9311938F5F8830D1F72F5F3F4F0E
:1008600028303105F9F464E070E080E090E00E9407
:10087000FC0511501F3F59F127C0C901B3E0880F93
:10088000991FBA95E1F7EC01CC5FDE4FDC01AC5B60
:10089000BE4FFC01EC57FE4F80E0C3CF402F20E05D
:1008A00030E0EBCFC901A3E0880F991FAA95E1F7CB
:1008B000EC01CC5FDE4FDC01AC5BBE4FFC01EC57C2
:1008C000FE4F80E0C5CF1FE120E030E0EBCFDF91AD
:1008D000CF911F910F910895CF93DF939927EC014A
:1008E000CC5FDE4FDC01AC5BBE4FFC01EC57FE4F32
:1008F00080E068834C9320838F5F28961896389603
:100900008830B9F7DF91CF9108951F920F920FB6FB
:100910000F921124AF92BF92CF92DF92EF92FF928B
:100920000F931F932F933F934F935F936F937F93F7
:100930008F939F93AF93BF93CF93DF93EF93FF93E7
:100940008FEC9EEF909385008093840060E089E0B7
:100950000E949706AA24BB247CC08881C81650F444
:1009600081E090E0022E02C0880F991F0A94E2F7FE
:100970008095D8228081C81650F481E090E0022E44
:1009800002C0880F991F0A94E2F78095E8228C91A3
:10099000C81650F481E090E0022E02C0880F991F23
:1009A0000A94E2F78095F8222F5F3F4F2196119627
:1009B00031962830310589F660E08AE00E9497067A
:1009C000FEBC0DB407FEFDCF8EB5EEBC0DB407FE28
:1009D000FDCF8EB5DEBC0DB407FEFDCF8EB581E038
:1009E00090E0002E02C0880F991F0A94E2F78EBD96
:1009F0000DB407FEFDCF8EB561E08AE00E94970638
:100A000060E08AE00E9497060F5F1F4F08301105D3
:100A100041F40894A11CB11C8FE1A816B104C9F4DB
:100A20001CC0C80133E0880F991F3A95E1F7EC012B
:100A3000CC5FDE4FDC01AC57BE4FFC01EC5BFE4FE0
:100A40002FEFD22E9FEFE92E8FEFF82E20E030E02F
:100A500084CFCA2C00E010E0E4CF61E089E00E947E
:100A60009706FF91EF91DF91CF91BF91AF919F9149
:100A70008F917F916F915F914F913F912F911F9136
:100A80000F91FF90EF90DF90CF90BF90AF900F90BD
:100A90000FBE0F901F9018951F920F920FB60F92D6
:100AA00011242F938F939F93AF93BF938091C8018D
:100AB0009091C901A091CA01B091CB018050904C96
:100AC000AF4FBF4F8093C8019093C901A093CA0153
:100AD000B093CB0127C08091C8019091C901A0912A
:100AE000CA01B091CB0180589E43A040B040809392
:100AF000C8019093C901A093CA01B093CB01809122
:100B0000CC019091CD01A091CE01B091CF01019681
:100B1000A11DB11D8093CC019093CD01A093CE0176
:100B2000B093CF018091C8019091C901A091CA01F1
:100B3000B091CB0181589E43A040B04060F6BF9178
:100B4000AF919F918F912F910F900FBE0F901F909B
:100B500018952FB7F8946091CC017091CD018091D8
:100B6000CE019091CF012FBF0895019751F0880FCA
:100B7000991F880F991F02972FB7F8940197F1F7E3
:100B80002FBF0895789484B5826084BD84B5816058
:100B900084BD85B5826085BD85B5816085BDEEE685
:100BA000F0E0808181608083E1E8F0E08081826014
:100BB0008083808181608083E0E8F0E080818160D3
:100BC0008083E1EBF0E0808184608083E0EBF0E003
:100BD000808181608083EAE7F0E0808184608083A7
:100BE0008081826080838081816080838081806851
:100BF00080831092C1000895EF92FF920F931F938C
:100C00007B018C018FB7F8944091CC015091CD01BC
:100C10006091CE017091CF018FBF2FB7F894809172
:100C2000CC019091CD01A091CE01B091CF012FBF09
:100C3000841B950BA60BB70B8E159F05A007B1075C
:100C400060F31F910F91FF90EF900895282F3327A5
:100C5000C90185579F4FFC01C895902D29583F4FDA
:100C6000F901C895802D882389F0E82FFF27E859DE
:100C7000FF4FC895E02DFF27662329F480819095CA
:100C80008923808308958081892B80830895482F4C
:100C90005527CA0181569F4FFC01C895202DCA01D6
:100CA00085579F4FFC01C895902D49585F4FFA0119
:100CB000C895302D332319F480E090E00895222365
:100CC00031F1233021F4809180008F7705C02430EA
:100CD00031F4809180008F7D8093800018C0213096
:100CE00019F484B58F7704C0223021F484B58F7D48
:100CF00084BD0DC0263021F48091B0008F7705C0EF
:100D0000273029F48091B0008F7D8093B000E32FCD
:100D1000FF27EE58FF4FC895E02DFF27808120E088
:100D200030E0892311F021E030E0C9010895482F17
:100D30005527CA0181569F4FFC01C895202DCA0135
:100D400085579F4FFC01C895902D49585F4FFA0178
:100D5000C895302D3323C9F1222331F1233021F4FA
:100D6000809180008F7705C0243031F4809180001D
:100D70008F7D8093800018C0213019F484B58F775F
:100D800004C0223021F484B58F7D84BD0DC026308F
:100D900021F48091B0008F7705C0273029F480912D
:100DA000B0008F7D8093B000E32FFF27E359FF4F02
:100DB000C895E02DFF27662329F48081909589232B
:100DC000808308958081892B808308956F927F921C
:100DD0008F929F92AF92BF92CF92DF92EF92FF924B
:100DE0000F931F93CF93DF93CDB7DEB739014A013D
:100DF00029893A894B895C89661977098809990993
:100E00002A193B094C095D090E94FD09E618F708FB
:100E100008091909A80197010E942F0A2A0D3B1DF4
:100E20004C1D5D1DCA01B901DF91CF911F910F913A
:100E3000FF90EF90DF90CF90BF90AF909F908F90FA
:100E40007F906F900895AF92BF92CF92DF92EF9212
:100E5000FF920F931F935B016C0161157105810572
:100E6000910529F460E070E080E090E01AC00E94F3
:100E7000D2077C010E94D2070027F7FC0095102FB3
:100E80008701FF24EE24AA2797FDA095BA2FE80E2C
:100E9000F91E0A1F1B1FC801B701A60195010E9478
:100EA0002F0A1F910F91FF90EF90DF90CF90BF908E
:100EB000AF900895EF92FF920F931F937B018C01E7
:100EC000621773078407950764F4261B370B480BDA
:100ED000590BCA01B9010E942307E60EF71E081F2D
:100EE000191FC801B7011F910F91FF90EF9008954E
:100EF000009711F00E94D7070895A0E0B0E0E3E862
:100F0000F7E00C94880AEC01A880B980CA80DB80E5
:100F1000A114B104C104D10449F482E4E82E8EEC9A
:100F2000F82E8CE0082F8FE1182F2EC0C601B501D6
:100F30002DE133EF41E050E00E942F0A27EA31E42F
:100F400040E050E00E94FD097B018C01C601B50123
:100F50002DE133EF41E050E00E942F0ACA01B901B0
:100F600024E13BE040E050E00E94FD09E61AF70A68
:100F7000080B190B17FF08C08FEF9FEFAFEFBFE70C
:100F8000E80EF91E0A1F1B1FE882F9820A831B83E1
:100F9000C7019F77EAE0CDB7DEB70C94A40A0E94A0
:100FA0007D07089580E091E00E947D070895AA27BB
:100FB000BB278093000190930101A0930201B0939D
:100FC000030108955058BB27AA270ED079C16AD1D2
:100FD00030F06FD120F031F49F3F11F41EF45FC167
:100FE0000EF4E095E7FB55C1E92F7BD180F3BA17EA
:100FF000620773078407950718F071F49EF593C193
:101000000EF4E0950B2EBA2FA02D0B01B901900123
:101010000C01CA01A0011124FF27591B99F0593F67
:1010200050F4503E68F11A16F040A22F232F342FAF
:101030004427585FF3CF469537952795A795F040FD
:101040005395C9F77EF41F16BA0B620B730B840B12
:10105000BAF09150A1F0FF0FBB1F661F771F881FCA
:10106000C2F70EC0BA0F621F731F841F48F4879522
:1010700077956795B795F7959E3F08F0B3CF939511
:10108000880F08F09927EE0F9795879508950CD053
:1010900017C10FD140F006D130F021F45F3F19F0B5
:1010A000F8C0511141C1FBC01CD198F39923C9F379
:1010B0005523B1F3951B550BBB27AA27621773075E
:1010C000840738F09F5F5F4F220F331F441FAA1F12
:1010D000A9F333D00E2E3AF0E0E830D091505040D2
:1010E000E695001CCAF729D0FE2F27D0660F771F80
:1010F000881FBB1F261737074807AB07B0E809F062
:10110000BB0B802DBF01FF2793585F4F2AF09E3FF6
:10111000510568F0BEC008C15F3FECF3983EDCF3B8
:10112000869577956795B795F7959F5FC9F7880F6F
:10113000911D9695879597F90895E1E0660F771FC1
:10114000881FBB1F621773078407BA0720F0621B52
:10115000730B840BBA0BEE1F88F7E095089504D04B
:101160006894B111E1C00895C4D088F09F5790F001
:10117000B92F9927B751A0F0D1F0660F771F881FBC
:10118000991F1AF0BA95C9F712C0B13081F0CBD0CF
:10119000B1E00895C8C0672F782F8827B85F39F06D
:1011A000B93FCCF3869577956795B395D9F73EF41B
:1011B00090958095709561957F4F8F4F9F4F0895C3
:1011C000E89409C097FB3EF49095809570956195E1
:1011D0007F4F8F4F9F4F9923A9F0F92F96E9BB2797
:1011E0009395F695879577956795B795F111F8CF13
:1011F000FAF4BB0F11F460FF1BC06F5F7F4F8F4F7E
:101200009F4F16C0882311F096E911C0772321F073
:101210009EE8872F762F05C0662371F096E8862F0B
:1012200070E060E02AF09A95660F771F881FDAF762
:10123000880F9695879597F9089507D008F481E06F
:10124000089503D008F48FEF0895990F0008550F03
:10125000AA0BE0E8FEEF16161706E807F907C0F03C
:1012600012161306E407F50798F0621B730B840B44
:10127000950B39F40A2661F0232B242B252B21F41E
:1012800008950A2609F4A140A6958FEF811D811DBE
:10129000089597F99F6780E870E060E008959FEFF8
:1012A00080EC089500240A941616170618060906FD
:1012B000089500240A9412161306140605060895CC
:1012C000092E0394000C11F4882352F0BB0F40F454
:1012D000BF2B11F460FF04C06F5F7F4F8F4F9F4F94
:1012E000089557FD9058440F551F59F05F3F71F016
:1012F0004795880F97FB991F61F09F3F79F087957D
:101300000895121613061406551FF2CF4695F1DF05
:1013100008C0161617061806991FF1CF8695710595
:10132000610508940895E894BB2766277727CB01C9
:1013300097F908950BD0C4CFB5DF28F0BADF18F0C5
:10134000952309F0A6CFABCF1124EECFCADFA0F3CF
:10135000959FD1F3950F50E0551F629FF001729F4A
:10136000BB27F00DB11D639FAA27F00DB11DAA1F69
:10137000649F6627B00DA11D661F829F2227B00DB6
:10138000A11D621F739FB00DA11D621F839FA00D41
:10139000611D221F749F3327A00D611D231F849F91
:1013A000600D211D822F762F6A2F11249F575040E8
:1013B0008AF0E1F088234AF0EE0FFF1FBB1F661F83
:1013C000771F881F91505040A9F79E3F510570F03C
:1013D00060CFAACF5F3FECF3983EDCF3869577951C
:1013E0006795B795F795E7959F5FC1F7FE2B880F37
:1013F000911D9695879597F90895629FD001739FE7
:10140000F001829FE00DF11D649FE00DF11D929FA0
:10141000F00D839FF00D749FF00D659FF00D9927DF
:10142000729FB00DE11DF91F639FB00DE11DF91F03
:10143000BD01CF011124089597FB092E07260AD07C
:1014400077FD04D027D006D000201AF4709561955E
:101450007F4F0895F6F7909581959F4F089597FBDC
:10146000092E05260ED057FD04D028D00AD0001C26
:1014700038F450954095309521953F4F4F4F5F4F31
:101480000895F6F790958095709561957F4F8F4FF1
:101490009F4F0895AA1BBB1B51E107C0AA1FBB1F8A
:1014A000A617B70710F0A61BB70B881F991F5A95F0
:1014B000A9F780959095BC01CD010895A1E21A2E5F
:1014C000AA1BBB1BFD010DC0AA1FBB1FEE1FFF1FE8
:1014D000A217B307E407F50720F0A21BB30BE40B38
:1014E000F50B661F771F881F991F1A9469F760957F
:1014F0007095809590959B01AC01BD01CF01089539
:101500002F923F924F925F926F927F928F929F9213
:10151000AF92BF92CF92DF92EF92FF920F931F9301
:10152000CF93DF93CDB7DEB7CA1BDB0B0FB6F894B2
:10153000DEBF0FBECDBF09942A88398848885F84F2
:101540006E847D848C849B84AA84B984C884DF8063
:10155000EE80FD800C811B81AA81B981CE0FD11D47
:101560000FB6F894DEBF0FBECDBFED010895FFCFDB
:041570000100000076
:00000001FF
